:03000000023A576A
:0C3A570078FFE4F6D8FD758165023A9E08
:1015830020000A3C2E2E2E3E004950436F6E6E659E
:1015930063745245510A004950436F6E6E6563741C
:1015A300000A49504E6F41434B210A003E432C56DB
:1015B3002C43432CC0E4E0EFF2E5F020D1E8EDEA60
:1015C300EEEC49500A003E432C4D41432C2530326A
:1015D30062583A25303262583A25303262583A25F9
:1015E300303262583A25303262583A2530326258E6
:1015F3002C4D414320E0E4F0E5F10A003E432C5634
:1016030045522C20332E3220EEF2202573202573F1
:101613002CC2E5F0F1E8FF20495020ECEEE4F3EBB7
:10162300FF0A0053657020313620323031300031EB
:10163300303A35303A3332003E432C4C442C50522E
:101643004F473A2020202020202020202020202027
:101653002020202020202020202020202020202087
:101663002020202020202020202020202020202077
:101673002020202020202020202020202020202067
:1016830020202020202020202CC4E0F2E020EFF0B6
:10169300EEF8E8E2EAE828F4E0E9EB290A003E2A5A
:1016A3002C312CCEF1EDEEE2EDFBE520EFE0F0E0A6
:1016B300ECE5F2F0FB20F1E5F2E5E2EEE3EE20E803
:1016C300EDF2E5F0F4E5E9F1E00A003E412C4130AA
:1016D300312C2562752E2562752E2562752E2562A5
:1016E300752C495020E0E4F0E5F120E0E4E0EFF26E
:1016F300E5F0E00A003E412C4130322C2562752E84
:101703002562752E2562752E2562752C495020E0C1
:10171300E4F0E5F120EEF1ED2E20F1E5F0E2E5F065
:10172300E00A003E412C4130332C2562752E2562A0
:10173300752E2562752E2562752C495020E0E4F044
:10174300E5F120F0E5E72E20F1E5F0E2E5F0E00A2F
:10175300003E412C4130342C2562752E2562752EB6
:101763002562752E2562752CCCE0F1EAE020F1E5C7
:10177300F2E80A003E412C4130352C2562752E25B6
:1017830062752E2562752E2562752CD8EBFEE70A4D
:10179300003E2A2C312CC4EEEF2E20EFE0F0E0ECDB
:1017A300E5F2F0FB20F1E5F2E5E2EEE3EE20E8ED11
:1017B300F2E5F0F4E5E9F1E00A003E422C53303162
:1017C3002C2562752CC6E4E0F2FC20E7E0EFF0EE96
:1017D300F1E020F1EEE5E4E8EDE5EDE8FF20EEF2DF
:1017E30020F1E5F0E2E5F0E00A003E422C5330320E
:1017F3002C2562752CCEE1ECE5ED20F120F1E5F02E
:10180300E2E5F0EEEC20E1E5E720EAE2E8F2E0EDE4
:10181300F6E8E90A003E422C5330332C2562752C3E
:10182300CFE5F0E5E7E0EFF3F1EA20EFF0E820EFB2
:10183300EEF2E5F0E520F1E2FFE7E820F120F1E543
:10184300F0E2E5F0EEEC0A003E422C5330382C2552
:1018530062752CCCE5E4EBE5EDEDFBE92049502086
:10186300EAE0EDE0EB28E7E0E4E5F0E6EAE020E497
:10187300EE203520F1E5EA290A003E454E440A00F0
:101883000A44756D705820202020203030203031DC
:101893002030322030332030342030352030362091
:1018A300303720303820303920304120304220304A
:1018B30043203044203045203046000A3A003A2085
:1018C300000A000A44756D70442020202020303027
:1018D3002030312030322030332030342030352056
:1018E3003036203037203038203039203041203016
:1018F300422030432030442030452030460045729A
:1019030072206B657900526420656570726F6D0A91
:10191300005264204D454D0A00526420436F6465B4
:101923000A00577269746520436F64650A00446551
:101933006275674950204F4E0A00446562756749D6
:1019430050204F46460A00446562756755736572B9
:10195300204F6E0A00446562756755736572204FA8
:1019630046460A0044656275674D7367204F6E0AE9
:101973000044656275674D7367204F46460A00430E
:101983006F6E666967206C6F636B210A0057722064
:10199300656570726F6D0A00205361766520656519
:1019A30070726F6D210A00457272204D4143210010
:1019B3004C6F61643E3E002A00CEF8E8E1EAE00A9B
:1019C30000202D202575282575290A003C4130313A
:1019D3003D003C4130323D003C4130333D003C4111
:1019E30030343D003C4130353D003C21003C533018
:1019F300313D003C5330323D003C5330333D003CDD
:101A03005330353D003C5330383D003C5330363D78
:011A130000D2
:06447200010B000109002E
:10446200C28E438910758BFF758DB7D2ABD28E2267
:03001B000239396E
:10393900C0E0C083C082C0D0C28E758BFF758DB7C1
:1039490020060675A61E75A6E10509D202E50B60DB
:1039590002050B050EE50E540F7051E50AD39401CB
:103969004002150AD20EE50E543F7012D20090663D
:103979008EE0600A04F0E0D394B44002D206906667
:1039890087E0600204F0906104E0600214F0906640
:103999008FE0D394014003E014F0300502050CE5F3
:1039A9000DD394644004D2068002050DE508D39432
:1039B9000140021508D28ED0D0D082D083D0E03217
:1008DF00C291C290D2B5C20B7D027C007F07124439
:1008EF002B8F47E547646060097D017F601243C627
:1008FF00D20BE4FDFC7F0B12442B8F47E54730E60C
:10090F00097D04E4FF1243EAD20B7D017C007F07CF
:10091F0012442B8F47E5477008FD7FFF1243C6D265
:10092F000B300B03126000C288C2A8C2AA758900DF
:10093F00123E0490633FE0B4FA06A3E064CE607BFE
:10094F00E4F54774372547F582E43463F583E4F023
:10095F000547E547B443EC90633F74FAF0A374CEB8
:10096F00F0A374CCF0906345740AF0E4A3F0A304F1
:10097F00F0A3F090633B74FFF0A3F0A3F0E4A3F0B7
:10098F009063567403F0E4F547E5472401FFE43321
:10099F00FE74372547F582E43463F583E0FD124397
:1009AF00A20547E547C3944340DFE4F5A775A61EAC
:1009BF0075A6E1907FF0F0A3F080FE90634A740378
:1009CF00F0A374CCF0E4906349F090668CF0A3F040
:1009DF00123399C2B51237D6C20612422AD20BC2AF
:1009EF000DC20C9065777408F09062B57424F0E432
:1009FF00A3F090633FE09062B7F0906340E09062A5
:100A0F00B8F0906341E09062B9F0906342E0906279
:100A1F00BAF0906343E09062BBF0906344E0906261
:100A2F00BCF0750A01E4906578F0C207C208C209EC
:100A3F00C20A200B18AF47FE7D0312347FE4FF126A
:100A4F0038897E157F83E4FBFDFC122FB690668EEE
:100A5F00E060037401F0E4906104F0F50C906576AA
:100A6F00F0F50D12446275A70775A61E75A6E1D2A3
:100A7F00AFE4F50D906104E07003120F6290668F82
:100A8F00E06401701D9080007410F09080A874FFD6
:100A9F00F0A3F0A3F0A3F0E490668FF0D20BC20C9A
:100AAF00C20D908008E0F54730E405D2077410F0CE
:100ABF00E54730E508D2099080087420F0E547300B
:100ACF00E608D2089080087440F0E50CC394034008
:100ADF0019908002E4F0908001F0908000F0E50C16
:100AEF0094064006E4F50C12422A9080A0E07003B1
:100AFF00123F749080B8E07003123E829080D0E075
:100B0F0070031241CE908000E07013300710123046
:100B1F00BD906332EFF0D394004003120026908013
:100B2F0002E07006908000E06005D205020A80C2E4
:100B3F0005E4F50C906104E06003020A80200B12BB
:100B4F00906579E0600C7E157F851232B1E4906577
:100B5F0079F0300912122BFE906332EFF0D394002C
:100B6F004005E0FF120022200803020D04122A772D
:100B7F00906332EFF07003020A80906376E054BF07
:100B8F00247F7003020C5F147003020C3724026081
:100B9F0003020CA6200B077E157F8C1232B1200F9B
:100BAF0003020D0490634EE07006906352E060679D
:100BBF00906683E0FF90634EE0B50724906684E073
:100BCF00FE90634FE0B50618906685E0FE90635087
:100BDF00E0B5060C906686E0FE906351E06E6037DC
:100BEF00906352E06F6003020D04906684E0FF9003
:100BFF006353E06F6003020D04906685E0FF90631E
:100C0F0054E06F6003020D04906686E0FF90635519
:100C1F00E06F6003020D04C2039065787401F01257
:100C2F00447C750A01020D0490668EE06003740126
:100C3F00F090667BE0FF906378E06F6003020D0435
:100C4F0090667BE004F0E4F50A906576F0020D04FF
:100C5F00300303020D04906345E07003020A809095
:100C6F0062B4E06008906356741EF080069063567D
:100C7F007403F012447AD203E4F50A906576F0908B
:100C8F00668704F0E490667AF0A3F0200B677E1578
:100C9F007F9A1232B1805E90668EE060037401F02D
:100CAF00300352906376E020E74B906378E0FF903B
:100CBF00667AE0FE6F600D906682E07007EE146F4B
:100CCF007033801390667AE004F0906332E0FFD3C4
:100CDF009404400312447B9060007482F0A374016B
:100CEF00F0906378E0906002F07E607F007D0312E9
:100CFF003B6A020A80200303020E22E50A706E127D
:100D0F0039C9EF60237E647F76906477E02404FD19
:100D1F00123B6A906682E07009906356E0F50A0212
:100D2F000A80E4F50A020A80906687E0D3943C407B
:100D3F003C906682E070369062B4E07030906687C7
:100D4F0004F0124479E4906476F0A37412F0906684
:100D5F007BE0906478F0A374FDF090610563A201CD
:100D6F0090647A63A2017F121227C5809812001E29
:100D7F008F47E547B401159060007483F0E4A3F04A
:100D8F007E607F007D02123B6A020A80E547D394A2
:100D9F0001401C9060007483F0A37401F0E54724B8
:100DAF00FEA3F07E607F007D03123B6A020A80E59E
:100DBF000A64016003020A80906576E004F0200B5C
:100DCF00077E157FA41232B1906356E0C3941E5074
:100DDF0004E02402F0906576E0C39405400DC20351
:100DEF00E4906578F012447C020A807C667D8390E3
:100DFF00634AE0FAA3E0FB7F02123D807E647F76B8
:100E0F00906477E02404FD123B6A906356E0F50A84
:100E1F00020A80E50A64016003020A80906578E0A7
:100E2F0014604624FE6042147003020F1524046000
:100E3F0003020A80E4F50C200F139065787404F018
:100E4F00906576E05401F0750A01020A80908002E5
:100E5F007410F0E4906578F090657604F0750A12DE
:100E6F0090668374FFF0020A80906683E07003023D
:100E7F000EFF9064767480F09064787401F0E4A3B0
:100E8F00F0A304F0A37430F0A3747BF0E4F547747F
:100E9F007D2547F582E43464F583747DF0747E25F7
:100EAF0047F582E43464F583E4F0E5472407906462
:100EBF0077F07C667D8390634AE0FAA3E0FB7F02C4
:100ECF00123D807E647F76E5472409FD123B6A90D0
:100EDF006682E0601B12447AD203E4F50A906576CD
:100EEF00F090668704F0E490667AF0A3F0020A802F
:100EFF00300F07E4906578F080069065787404F001
:100F0F00750A12020A809080027410F0750A03901D
:100F1F006576E06401FFF09065787401F0EF701969
:100F2F00906352E06013FCA3E0FDA3E0FEA3E0FF9B
:100F3F00906683122359020A8090634EE0FCA3E06F
:100F4F00FDA3E0FEA3E0FF906683122359020A80FF
:020F5F0080FE12
:010F6100226D
:10002600906377E0B444047F0180027F009063769A
:10003600E0B447047E0180027E00EE5F604A906372
:100046003FE0906378F0906340E0906379F09063CE
:1000560041E090637AF0906342E090637BF09063B6
:1000660043E090637CF0906344E090637DF090639E
:10007600777452F09062AE63A2019080A863A201E9
:100086007F061227C50208D5906332E0C394085054
:10009600030208DE90633FE0FF906378E06F600341
:1000A6000208DE906340E0FF906379E06F60030230
:1000B60008DE906341E0FF90637AE06F6003020818
:1000C600DE906342E0FF90637BE06F60030208DE30
:1000D600906343E0FF90637CE06F60030208DE906C
:1000E6006344E0FF90637DE06F60030208DE906387
:1000F60077E06444701A9080A8E0B4FF139062AE73
:1001060063A2019080A863A2017F061227C5801012
:100116009062B2E09080ACF09062B3E09080ADF077
:1001260090668EE060037401F090668F7464F090C0
:1001360063777452F0906376E0646D600302027830
:100146007BFF7A1579AF121E817BFF7A1579C990EC
:10015600633FE0F550A3E0F551A3E0F552A3E0F5C7
:1001660053A3E0F554A3E0F555121E817550FF75B3
:1001760051167552267553FF7554167555327BFF09
:100186007A1579FF121E817BFF7A16793B121E8142
:100196007BFF7A1679A1121E817BFF7A1679CE90A3
:1001A6006345E0F550A3E0F551A3E0F552A3E0F571
:1001B60053121E817BFF7A1679F890634EE0F55054
:1001C600A3E0F551A3E0F552A3E0F553121E817B9F
:1001D600FF7A177926906352E0F550A3E0F551A314
:1001E600E0F552A3E0F553121E817BFF7A1779548E
:1001F60090633BE0F550A3E0F551A3E0F552A3E090
:10020600F553121E817BFF7A177977906337E0F5F5
:1002160050A3E0F551A3E0F552A3E0F553121E8179
:100226007BFF7A177994121E817BFF7A1779BDA21C
:100236000FE433F550121E817BFF7A1779ED906635
:1002460082E0F550121E817BFF7A18791890668E2F
:10025600E0F550121E817BFF7A18794B9062B4E06C
:10026600F550121E81122D6F7BFF7A18797D121EB2
:100276008122906376E0644C70737E187F83FBFD69
:10028600FC122FB690637EE0F548A3E0F549E4F54D
:100296004BE548906380F0A3E549F07E187FBE7C6D
:1002A600637D807B02122FB6E4F54A854982854834
:1002B60083E0FF7480254AF582E43463F583EFF02A
:1002C6000549E54970020548054AE54AB410DC7E51
:1002D600187FC17C637D807B10122FB6054BE54BE2
:1002E600C3941040AC7E187FC41232B1229063765C
:1002F600E0646C7060F54C7E187FC6FBFDFC122F27
:10030600B6E4F54BE4906380F0A3E54CF07E187FED
:10031600BE7C637D807B02122FB6E4F54AA84CE6CC
:10032600FF7480254AF582E43463F583EFF0054CCB
:10033600054AE54AB410E67E187FC17C637D807B62
:1003460010122FB6054BE54BC3940840B77E187FB5
:10035600C41232B122906376E0644B7061F54A7440
:1003660068254AF582E43463F583E06032746825D3
:100376004AF582E43463F583E0F460237468254A21
:10038600F582E43463F583E0FF747E254AF582E462
:100396003463F583E0B50710054AE54AB408C09012
:1003A60061047432F00208D59063767421F0300B44
:1003B600030208D57E197F011232B10208D5906377
:1003C60076E0B4521A200B077E197F091232B190DB
:1003D60063767472F07E637F767D08123AE322902C
:1003E6006376E064497045200B077E197F1412324C
:1003F600B190637EE0F548A3E0F549E4F54A854906
:1004060082854883E0FF7480254AF582E43463F5EB
:1004160083EFF00549E54970020548054AE54AB407
:1004260080DC7E637F767D8A123AE322906376E0F3
:1004360064437046200B077E197F1C1232B190630D
:100446007EE0F548A3E0F549E4F54A85498285480A
:1004560083E493FF7480254AF582E43463F583EFE1
:10046600F00549E54970020548054AE54AB480DBCE
:100476007E637F767D8A123AE322906376E0645A41
:100486007053200B077E197F251232B190637EE0F0
:10049600F548A3E0F5497C637D807B80AF49AE4893
:1004A600124348E4F54A854982854883E493FF74FC
:1004B60080254AF582E43463F583EFF00549E54982
:1004C60070020548054AE54AB480DB7E637F767D87
:1004D6008A123AE322906376E06444600302056C74
:1004E60090637EE0FF644470030208D5EFB4310CDC
:1004F600C20B7E197F311232B10208D590637EE0BD
:10050600B4300CD20B7E197F3D1232B10208D59061
:10051600637EE0B4320CD20C7E197F4A1232B102ED
:1005260008D590637EE0B4330CC20C7E197F581256
:1005360032B10208D590637EE0B4340CD20D7E1938
:100546007F671232B10208D590637EE0B4350CC2E3
:100556000D7E197F741232B10208D590637EE0FFDA
:100566001200210208D5906104E07013200B077E6B
:10057600197F821232B19063767421F00208D59009
:1005860061047432F0906376E0FFB45104C2AF8028
:10059600FEEF64577045200B077E197F901232B12B
:1005A60090637FE0906332F0E4F54A906332E0FFB7
:1005B600E54AC39F40030208D57480254AF582E4C4
:1005C6003463F583E0FF90637EE0254A24ADF5822F
:1005D600E43461F583EFF0054A80D0906376E064F9
:1005E60053600302068F200B077E197F9B1232B1E0
:1005F60090633FE0FF9061B6E06F703C906340E02F
:10060600FF9061B7E06F7030906341E0FF9061B892
:10061600E0B50724906342E0FF9061B9E0B50718A2
:10062600906343E0FF9061BAE0B5070C906344E045
:10063600FF9061BBE06F60169063767421F0300B1B
:10064600030208D57E197FAA1232B10208D5E4F555
:100656004AE4F50DAF4AFE74AD254AF582E43461ED
:10066600F583E0FD1243A2054AE54AC394FE40E144
:10067600C2AFE4907FF0F0A3F0907FFD74AAF0A3E0
:1006860074FFF0A37455F080FE906376E0644F70BB
:100696005A90637EE0F548A3E0F549E54945487080
:1006A6000A200B077E197FB31232B1200B077E1981
:1006B6007FBA1232B1E4F54A7480254AF582E434F1
:1006C60063F583E0854982854883F00549E54970ED
:1006D600020548054AE54AB480DE90668DE024802E
:1006E600F090668CE03400F00208D5906376E06402
:1006F60045707490637EE0FEA3E0FF907FF0EEF01D
:10070600A3EFF0D39400EE94044038907FF0E0FE1F
:10071600A3E0FF90668CE0FCA3E0FD9FEC9E4023E7
:10072600E42FFFEE3401FED3ED9FEC9E5015C2AFD1
:10073600907FFD74AAF0A374FFF0A37455F0E4F55E
:10074600A780FE7E197FBC1232B17BFF7A1979C46D
:10075600907FF0E0F550A3E0F55190668CE0F552FD
:10076600A3E0F553121E81906376E0646560030290
:1007760008DE90637EE0FFA3E0907FF0CFF0A3EF6A
:10078600F0E4F548F549D3907FF1E09549907FF084
:10079600E095484020E4F50D2549FFE5483401FE83
:1007A600854982854883E0FD1243A20549E54970E3
:1007B60002054880D17E197FCF123BF1EF4E6020B3
:1007C600120003906345EFF0120003906346EFF0CA
:1007D600120003906347EFF0120003906348EFF0B6
:1007E6007E197FD5123BF1EF4E6020120003906315
:1007F6004EEFF012000390634FEFF0120003906388
:1008060050EFF0120003906351EFF07E197FDB1278
:100816003BF1EF4E6020120003906352EFF012009E
:1008260003906353EFF0120003906354EFF012004D
:1008360003906355EFF07E197FE1123BF1EF4E60B6
:100846002012000390633BEFF012000390633CEF2D
:10085600F012000390633DEFF012000390633EEF49
:10086600F07E197FE7123BF1EF4E602012000390F5
:100876006337EFF0120003906338EFF01200039035
:100886006339EFF012000390633AEFF0E4F54AE4BF
:10089600F50DE54A2401FFE433FE7437254AF58257
:1008A600E43463F583E0FD1243A2054AE54AC394A6
:1008B6004340DCC2AFE4907FF0F0A3F0907FFD747C
:1008C600AAF0A374FFF0A37455F0E4F5A780FE7EAA
:0808D600637F767D08123AE30E
:0108DE0022F7
:10431000AE07EEC39430400BEED394395005EE2433
:10432000D0FF22EEC39461400BEED394665005EEAD
:1043300024A9FF22EEC39441400BEED394465005CE
:08434000EE24C9FF22AF0622A2
:104448009062ADE004F070069062ACE004F0906217
:0A445800ACE0FEA3E0FF12440E22C8
:10000300124448124310EFC454F0FEC00612444891
:08001300124310D0E02FFF2280
:10417100E4906B60F0124448906B61EFF0C39430AF
:104181004018E0FFD394395011906B60E02405F59D
:1041910082E43461F583EFF08011906B60E02405D7
:1041A100F582E43461F583E4F0800C906B60E00407
:1041B100F0E0D3940840BE754D00754E00754F0078
:0C41C100E4F5507B017A6179051228D3E7
:0141CD0022CF
:043BF1008E4D8F4E18
:103BF5009062ACE4F0A374FFF0124448EF606EF4F9
:103C0500606B854E82854D83E493B507EC754F0156
:103C1500E54E254FF582E4354DF583E49360259017
:103C250062ADE0254FFF9062ACE03400FE12440E19
:103C3500E54E254FF582E4354DF583E493B507044C
:103C4500054F80CCE54E254FF582E4354DF583E4EF
:103C55009370A6E54F24FFFFE434FFFE9062ADE0CC
:103C65002FF09062ACE03EF07E007F0122E4FEFF83
:013C7500222C
:103399007E197FED123BF1EF4E70037F01227E19FA
:1033A9007FF0123BF1EF4E600C124448EF24D02419
:1033B900FF920F8002D20F7E197FF6123BF1EF4E7A
:1033C900600C124448EF24D0906682F08005E490A6
:1033D9006682F07E197FFC123BF1EF4E600C1244BD
:1033E90048EF24D090668EF08005E490668EF07EDA
:1033F9001A7F02123BF1EF4E600C124448EF24D0C1
:1034090024FF92018002C2017E1A7F08123BF1EF6C
:103419004E600C124448EF24D09062B4F08005E469
:103429009062B4F090633F63A20190667C63A2014D
:103439007F061227C530013B7E1A7F0E123BF1EF42
:103449004E603012000390667CEFF0120003906624
:103459007DEFF012000390667EEFF0120003906694
:103469007FEFF0120003906680EFF0120003906680
:0634790081EFF07F00224C
:10428400906577E0C3947C40027F0A906577E0FEF6
:1042940004F074B52EF582E43462F583EFF0BF0ABE
:1042A40027906577E0FF04F074B52FF582E434625B
:1042B400F583E4F0906577E0FF123C7690657774BF
:0942C40008F09062B6E004F0225B
:10422A009080007480F090633763A201F583F58271
:10423A0063A2017F081227C590633F63A2019080A1
:10424A008863A2017F0A1227C59080927407F0A39F
:10425A0074D0F0A37406F0906349E0FF9080B1F047
:10426A009080E1EFF09080957455F0A3F090800073
:0A427A007401F090800974F0F02246
:103F7400908009E04410F09080A0E070609080A1EF
:103F84007482F09080A874FFF0A3F0A3F0A3F07FF4
:103F9400039080AEEFF0A374CBF09080007402F035
:103FA400906B5412236500000000906B54E09080E5
:103FB40040F0906B55E0908041F0906B56E090801B
:103FC40042F0906B57E0908043F0A3E4F0A3F0A399
:0D3FD400F0A3F0908018F0A3F0A3F0A3F08C
:013FE10022BD
:1041CE00908009E04440F09080D17482F07F03909B
:1041DE0080DEEFF0A374CCF09080027402F0906B4E
:1041EE005812236500000000906B58E0908058F044
:1041FE00906B59E0908059F0906B5AE090805AF095
:10420E00906B5BE090805BF0A3E4F0A3F0A3F0A3CF
:0B421E00F0908030F0A3F0A3F0A3F0BC
:014229002272
:103E8200908009E04420F09080B8E0706C9080B996
:103E92007482F07F039080C6EFF07FCDA3EFF07FB6
:103EA200039080C4EFF0A374CDF09080C074FFF053
:103EB200A3F0A3F0A3F09080017402F0906B5C1267
:103EC200236500000000906B5CE090804CF0906BEA
:103ED2005DE090804DF0906B5EE090804EF0906BD4
:103EE2005FE090804FF0A3E4F0A3F0A3F0A3F09082
:093EF2008024F0A3F0A3F0A3F07A
:013EFB0022A4
:103D80008C488D49A907EAFDE975F018A424ACFF19
:103D9000E5F034808F82F583EDF0EBFDE975F018E6
:103DA000A4FFAEF024ACFBEE34808B82F583A3ED50
:103DB000F08549828C83E0FDEF24A8FFEE3480FE7D
:103DC0008F82F583EDF08549828C83A3E08F828E0C
:103DD00083A3F0854982854883A3A3E0FDE975F0BC
:103DE00018A424A8FFE5F03480FE8F82F583A3A3F6
:103DF000EDF08549828C83A3A3A3E08F828E83A3F9
:043E0000A3A3F02266
:063AE3008D4DAB07AA06A1
:103AE900908000E030E5079065797401F022906BD1
:103AF90054E0FCA3E0FDA3E0FEA3E0F5518E508D58
:103B09004F8C4EAE02AF038E838F8263A201E550C4
:103B1900540744C0F58385518263A201AF4D122831
:103B290037E4FCFDFEE551254DF551EE3550F550D4
:103B3900ED354FF54FEC354EF54E908040E54EF0A2
:103B4900A3E54FF0A3E550F0A3E551F09080007490
:103B590020F0AF51AE50AD4FAC4E906B541223597B
:013B69002239
:063B6A008D48AB07AA061E
:103B7000908002E030E5079065797403F022906B45
:103B800058E0FCA3E0FDA3E0FEA3E0F54C8E4B8DD6
:103B90004A8C49AE02AF038E838F8263A201E54B4C
:103BA000540744D0F583854C8263A201AF481228A4
:103BB00037E4FCFDFEE54C2548F54CEE354BF54B66
:103BC000ED354AF54AEC3549F549908058E549F01C
:103BD000A3E54AF0A3E54BF0A3E54CF09080027416
:103BE00020F0AF4CAE4BAD4AAC49906B5812235904
:013BF00022B2
:023889008F4866
:10388B00908001E030E5099065797402F07F0022A9
:10389B00906B5CE0FCA3E0FDA3E0FEA3E0F54C8E97
:1038AB004B8D4A8C4990667C63A201E54B540744CF
:1038BB00C8F583854C8263A2017F0612284DE54C27
:1038CB002406F54CE4354BF54BE4354AF54AE43523
:1038DB0049F54990657A63A201E54B540744C8F555
:1038EB0083854C8263A201AF4812284DE4FCFDFE98
:1038FB00E54C2548F54CEE354BF54BED354AF54A85
:10390B00EC3549F54990804CE549F0A3E54AF0A325
:10391B00E54BF0A3E54CF09080017420F0AF4CAE7A
:0D392B004BAD4AAC49906B5C122359AF487C
:01393800226C
:1030BD009081E0E0F5480548054805480548054874
:1030CD0005480548054805480548908010E0F54B32
:1030DD00A3E0F54CA3E0F54DA3E0F54E9081E1E0C2
:1030ED00F54805480548054805480548054805487B
:1030FD00054805480548908014E0F54FA3E0F550CC
:10310D00A3E0F551A3E0F552E551B54D08E552B5F3
:10311D004E037F0022E4F548E551540744E0F58362
:10312D0085528263A20190637663A2017F08122803
:10313D007D90637863A2019062AE63A2017F061257
:10314D0027C5906376E0F549A3E0F54AE4F548908C
:10315D006376E0702AA3E024F8F548E5515407445E
:10316D00E0F58385528274082582F582E43583F576
:10317D008363A20190637663A201AF4812287DAEEE
:10318D0049E4FCFDE552254AF552E5513EF551ED78
:10319D003550F550EC354FF54F908014E54FF0A3B9
:1031AD00E550F0A3E551F0A3E552F0908000744096
:0331BD00F0AF4828
:0131C00022EC
:102A77009081E6E0F54805480548054805480548BA
:102A870005480548054805480548908028E0F54B66
:102A9700A3E0F54CA3E0F54DA3E0F54E9081E7E008
:102AA700F5480548054805480548054805480548C7
:102AB70005480548054890802CE0F54FA3E0F55000
:102AC700A3E0F551A3E0F552E4F548E551B54D0A09
:102AD700E552B54E05C208022BE3E551540744F011
:102AE700F58385528263A20190637663A2017F0812
:102AF70012287D906376E0F549A3E0F54AE54A455B
:102B07004970099080027410F07F0022906683E07C
:102B1700FFF46030906378E06F6003022BAA906641
:102B270084E0FF906379E06F7079906685E0FF90AD
:102B3700637AE06F706D906686E0FF90637BE06F6D
:102B47006031805F906378E0906683F0906379E00E
:102B5700906684F090637AE0906685F090637BE0FE
:102B6700906686F090637CE0FFA3E090634ACFF025
:102B7700A3EFF0906376E0702AA3E024F8F548E528
:102B870051540744F0F58385528274082582F582F3
:102B9700E43583F58363A20190637663A201AF48AE
:102BA70012287DAE49E4FCFDE552254AF552E55170
:102BB7003EF551ED3550F550EC354FF54FAF4EAE74
:102BC7004DAD4CAC4BAB52AA51A950A84FD31223D1
:102BD7004840099080027410F07F002290802CE515
:102BE7004FF0A3E550F0A3E551F0A3E552F0908034
:062BF700027440F0AF483B
:012BFD0022B5
:102BFE009081E3E0F5480548054805480548054835
:102C0E000548054805480548054890801CE0F54BE9
:102C1E00A3E0F54CA3E0F54DA3E0F54E9081E4E082
:102C2E00F54805480548054805480548054805483E
:102C3E00054805480548908020E0F54FA3E0F55083
:102C4E00A3E0F551A3E0F552E4F548E551B54D0A80
:102C5E00E552B54E05C209022D54E551540744E81C
:102C6E00F58385528263A20190600463A2017F0EF8
:102C7E00122893906004E0F549A3E0F54A90600CA9
:102C8E00E0FFF4604A90667CE0FEEF6E7079A3E0A0
:102C9E00FF90600DE06F706F90667EE0FF90600EAB
:102CAE00E06F706390667FE0FF90600FE06F70578B
:102CBE00906680E0FF906010E06F704B906681E050
:102CCE00FF906011E06F703FE4906013F080089009
:102CDE00601374FFF0D2D9906004E0702AA3E02450
:102CEE00F2F548E551540744E8F583855282740E97
:102CFE002582F582E43583F58363A2019060046337
:102D0E00A201AF48122893AE49E4FCFDE552254AD4
:102D1E00F552E5513EF551ED3550F550EC354FF588
:102D2E004FAF4EAE4DAD4CAC4BAB52AA51A950A8C5
:102D3E004FD31223485006E54A4549700990800149
:102D4E007410F07F0022908020E54FF0A3E550F044
:102D5E00A3E551F0A3E552F09080017440F0AF4826
:012D6E002242
:0432B1008E4D8F4E61
:1032B500908000E030E5079065797401F022906B0D
:1032C50054E0FCA3E0FDA3E0FEA3E0F5548E538D8E
:1032D500528C51E554FFE5535407FEE42FF550EEAB
:1032E50034C0F54F855082F5837423F00550E550C1
:1032F5007002054F534FC7F582854F83740AF00559
:1033050050E5507002054F534FC790633F63A201CC
:10331500854F8385508263A2017F06122837740684
:103325002550F550E4354FF54F854D83854E826325
:10333500A201854F8385508263A20112281BE4FCFC
:10334500FDFE906B54E0F8A3E0F9A3E0FAA3E02FAB
:10335500FFEE3AFEED39FDEC38FCEF2408FFE43EC4
:10336500FEE43DFDE43CFC906B54122359906B54F4
:10337500E0908040F0906B55E0908041F0906B5666
:10338500E0908042F0906B57E0908043F090800091
:033395007420F0B1
:013398002212
:0A2FB6008E4D8F4E8C4F8D508B51C5
:102FC000908000E030E5079065797401F022906B05
:102FD00054E0FCA3E0FDA3E0FEA3E0F5578E568D80
:102FE000558C54E557FFE5565407FEE42FF553EE94
:102FF00034C0F552855382F5837423F00553E553AD
:10300000700205525352C7F582855283740AF00547
:1030100053E553700205525352C790633F63A201B8
:1030200085528385538263A2017F06122837740676
:103030002553F553E43552F552854D83854E826311
:10304000A20185528385538263A20112281B8F58E7
:10305000EF2553F553E43552F552E5516017854F8E
:103060008385508263A20185528385538263A201C6
:10307000AF51122837E55824082551F551FFE4FCDB
:10308000FDFEE5572FF557EE3556F556ED3555F55E
:1030900055EC3554F554908040E554F0A3E555F0D7
:1030A000A3E556F0A3E557F09080007420F0AF57E9
:0C30B000AE56AD55AC54906B5412235931
:0130BC0022F1
:06363C008E498F4A8D4B00
:10364200908000E030E5079065797401F022906B7C
:1036520054E0FCA3E0FDA3E0FEA3E0F5518E508D03
:103662004F8C4EE551FFE5505407FEE42FF54DEE29
:1036720034C0F54C854D82F5837423F0054DE54D3C
:103682007002054C534CC7F582854C83EBF0054D17
:10369200E54D7002054C534CC790633F63A2018510
:1036A2004C83854D8263A2017F061228377406255A
:1036B2004DF54DE4354CF54C854983854A8263A22C
:1036C20001854C83854D8263A201AF4B122837746A
:1036D20008254BF54BFFE4FCFDFEE5512FF551EEBD
:1036E2003550F550ED354FF54FEC354EF54E908097
:1036F20040E54EF0A3E54FF0A3E550F0A3E551F00D
:103702009080007420F0AF51AE50AD4FAC4E906B34
:0437120054122359D1
:013716002290
:023C76008F615C
:103C7800908000E030E5079065797401F022906B40
:103C880054E0FCA3E0FDA3E0FEA3E0F5658E648D9F
:103C9800638C62E565FFE5645407FEE42FFFEE34AC
:103CA800C09062B563A201F5838F8263A201AF6100
:103CB800122837E4FCFDFEE5652561F565EE3564FF
:103CC800F564ED3563F563EC3562F562908040E5A7
:103CD80062F0A3E563F0A3E564F0A3E565F09080E6
:103CE800007420F0AF65AE64AD63AC62906B5412A3
:023CF80023594E
:013CFA0022A7
:06347F008E4B8F4CAB05E3
:10348500908000E030E5079065797401F022906B3B
:1034950054E0FCA3E0FDA3E0FEA3E0F5528E518DC0
:1034A500508C4FE552FFE5515407FEE42FF54EEEE3
:1034B50034C0F54D854E82F5837423F0054EE54EF7
:1034C5007002054D534DC7F582854D83EBF0054ED2
:1034D500E54E7002054D90633F63A201854D8385DE
:1034E5004E8263A2017F061228377406254EF54EDB
:1034F500E4354DF54D534DC7E54B854E82854D83DE
:10350500F0054EE54E7002054D534DC7F582854DCC
:1035150083E54CF0054EE54E7002054D534DC7E56C
:1035250052240AF552E43551F551E43550F550E48D
:10353500354FF54F908040E54FF0A3E550F0A3E5FA
:1035450051F0A3E552F09080007420F0AF52AE51D7
:0A355500AD50AC4F906B5412235997
:01355F002249
:10404B00908009E04480F09080E97441F07F099002
:10405B0080F6EFF0A37464F09080037402F090800C
:10406B0003E020E1F9906A501223650000000090F4
:10407B006A50E0908064F0906A51E0908065F09017
:10408B006A52E0908066F0906A53E0908067F0A3EC
:10409B00E4F0A3F0A3F0A3F090803CF0A3F0A3F026
:0240AB00A3F080
:0140AD0022F0
:103560009081E9E0F54905490549054905490549BD
:1035700005490549054905490549908034E0F54A62
:10358000A3E0F54BA3E0F54CA3E0F54D9081EAE014
:10359000F5490549054905490549054905490549CB
:1035A000054905490549908038E0F54EA3E0F54FFF
:1035B000A3E0F550A3E0F551E550B54C08E551B551
:1035C0004D037F0022AF51AE50AD4FAC4EAB4DAA74
:1035D0004CA94BA84AD3122348400AAF51AE4DEE36
:1035E0009FF549800AAF51EFF404AE4D2EF549E541
:1035F00050540744E0F58385518263A201906A54D8
:1036000063A201AF491228ABE4FCFDFEE551254958
:10361000F551EE3550F550ED354FF54FEC354EF593
:103620004E908038E54EF0A3E54FF0A3E550F0A3AF
:0B363000E551F09080037440F0AF49BA
:01363B00226C
:0231C1008F4934
:1031C3009080E8E0640660037FFF22906A50E0FC91
:1031D300A3E0FDA3E0FEA3E0F54D8E4C8D4B8C4A9E
:1031E300E4FFFEFDFCAB4DAA4CA94BA84AC3122336
:1031F3004870609081F9E0F54A906A50E0FCA3E0E2
:10320300FDA3E0FEA3E0FFE4FAF9F8EF2401FFEAEF
:103213003EFEE93DFDE83CFC906A50122359906A5A
:1032230050E0FCA3E0FDA3E0FEA3E0FFE4F8EF24FD
:1032330001FFEA3EFEE93DFDE83CFC906A501223A3
:1032430059908064E0F54AA3E0F54BA3E0F54CA365
:10325300E0F54D906A5463A201E54C540744D8F558
:1032630083854D8263A201AF49122865E4FCFDFE0C
:10327300E54D2549F54DEE354CF54CED354BF54B0C
:10328300EC354AF54A908064E54AF0A3E54BF0A398
:10329300E54CF0A3E54DF09080037420F0AF4DAE04
:0D32A3004CAD4BAC4A906A501223597F008D
:0132B00022FB
:10440E00A2AF9210C2AF438E2075D2028F828E83DE
:0C441E00E0FFE4F5D2538EDFA21092AF55
:01442A00226F
:1043A200E5D220E0FBA2AF9210C2AF43D2028F82CD
:1043B2008E83EDF075D25063D250A21092AFE5D247
:0343C20020E0FBFD
:0143C50022D5
:103E0400E4FDED2401FFE433FE12440E74372DF576
:103E140082E43463F583EFF00DBD3FE6E4FDED2469
:103E24007FFFE433FE12440E742D2DF582E43461D9
:103E3400F583EFF0742D2DF582E43461F583E070A1
:103E44001B742D2DF582E43461F5837420F0742EF7
:103E54002DF582E43461F583E4F080040DBD80BE69
:103E6400E49061ACF0FDEDFF7E0012440E74AD2DC4
:0D3E7400F582E43461F583EFF00DBDFEE949
:013E8100221E
:024348008B4D9B
:10434A00A2AF9210C2AF85A24E53A2FE8E838F8275
:10435A0005A28C838D8274091228C1E54D53A2FEF1
:10436A0043A2201228C353A2DF854EA2A21092AF05
:01437A00FF43
:01437B00221F
:10442B00A2AF9210C2AF8C838D82EF1228C143A230
:0C443B00201228C353A2DFA21092AFFF92
:014447002252
:0243C6008F481E
:1043C800A2AF9210C2AFE4F5838D8274061228C1A1
:1043D800E54843A2201228C353A2DFA21092AF7F60
:0143E80001D3
:0143E90022B1
:0243EA008F48FA
:1043EC00A2AF9210C2AFE4F5838D82740A1228C179
:1043FC00E54843A2201228C353A2DFA21092AF7F3C
:01440C0001AE
:01440D00228C
:1026EA00A907E7FFA805EF93C3966008403B74FC6F
:1026FA002FFF80F00F08EF93C3966008402B74FBFE
:10270A002FFF80E00F08EF93C3966008401B74FA0E
:10271A002FFF80D00F08EF93D3966008400B74F90F
:10272A002FFF80C01F1F1F1F1FEF54FEF80303F760
:10273A00E893FC08E893FD08E893FE08E893FF2273
:10274A0009E993C39D6008402974FB29F980F109BE
:10275A00E993C39E6008401A74FA29F980E209E9EC
:10276A0093D39F6008400B74F929F980D31919197A
:10277A001919E9C313C313FF22740093F8ECC39821
:10278A004024701F740193F8EDC3984019701474B3
:0E279A000293F8EEC398400E7009740393F892
:1027A800EFC39840037F00227F0122EDF8E6F0088E
:1027B800A3DFFA22EDF8E0F608A3DFFA22E0A3632C
:1027C800A201F0A363A201DFF475A2002263A201B3
:1027D800F0A363A20122E0A363A201F0A363A20114
:1027E800E0A363A201F0A363A201E463A201F0A342
:1027F80063A201DFE175A20022E0A363A2016DFEDE
:10280800936CFDEE058393FC158363A201DFEA75E3
:10281800A200227F00E493A363A201F00F600CA33F
:10282800E583C2E3F58363A20180EA75A20022E092
:10283800A363A201F0A3E583C2E3F58363A201DFEA
:10284800EE75A20022E0A363A201F0A3E583C2E42F
:10285800D2E3F58363A201DFEC75A20022E0A36353
:10286800A201F0A3E58344F8C2E5F58363A201DF82
:10287800EC75A20022E583C2E3F583E0A363A2011D
:10288800F0A363A201DFEE75A20022E583C2E4D2C1
:0A289800E3F583E0A363A201F0A3BF
:1028A20063A201DFEC75A20022E58344F8F583E020
:1028B200A363A201F0A363A201DFEE75A20022F9D5
:1028C20022C002C004C00612FFF0D006D004D0021B
:0128D20022E3
:102463003E2A2C312CCFE0F0E0ECE5F2F0FB20F833
:10247300E8EDFB2043414E0A003E4C2C6B30312CDF
:1024830025732C43EAEEF0EEF1F2FC20EDE020F8A8
:10249300E8EDE52043414E2C30202D20353030EA45
:1024A300E1283530EC292C31202D203530EAE12884
:1024B300353030EC290A0030202D20353030EAE168
:1024C300283530EC290031202D203530EAE128353C
:1024D3003030EC29003E2A2C312CCFE0F0E0ECE543
:1024E300F2F0FB20EFF0EEF2EEEAEEEBE0204654E2
:1024F300330A003E4C2C4930312C256C752CD1EA23
:10250300EEF0EEF1F2FC20EEE1ECE5EDE02C313201
:1025130030302C323430302C343830302C393630A3
:10252300302C31393230300A003E532C4931322CB1
:102533002562752CC0E4F0E5F120E1EBEEEAE02042
:10254300D2C8D220EDE020F8E8EDE50A003E532C96
:102553006D2562752C25732CCFF0E8E1EEF0202574
:1025630062752028C0E4F0E5F120E820EFE0F0E018
:10257300ECE5F2F0FB290A003E532C5630382C25AB
:10258300752CCFE0F3E7E020E220EEEFF0EEF1E090
:10259300F528ECF1290A003C6B30313D003C493011
:1025A300313D003C4931323D003C5630383D000A54
:1025B30043616E45724749543A002043616E457248
:1025C30072434821000A000A5265713A00496E6954
:1025D300745443500A004C697374656E5443500A33
:1025E30000534F434B5F5443505F45535441424C58
:1025F30049534845440A000A2D3E20000A3C2D2039
:1026030000203C20000ACEF8E8E1EAE020CAD131FC
:1026130021000ACEF8E8E1EAE020CAD13221000A1B
:10262300CEF8E8E1EAE020CAD13321000ACEF8E887
:10263300E1EAE020CAD13421000ACEF8E8E1EAE079
:1026430020CAD13521000ACEF8E8E1EAE020CAD158
:102653003621000ACEF8E8E1EAE020CAD1372100AA
:102663000A455252210A003C6D303D000000003CF7
:102673006D313D000000003C6D323D000000003C28
:102683006D333D000000003C6D343D000000003C14
:102693006D353D000000003C6D363D000000003C00
:1026A3006D373D000000003C6D383D000000003CEC
:1026B3006D393D000000003C6D31303D0000003CB1
:1026C3006D31313D0000003C6D31323D0000003C76
:1026D3006D31333D0000003C6D31343D0000003C62
:0726E3006D31353D000000E0
:0100210022BC
:03002300023CFBA1
:0B3CFB00C0E0C083C082C0D075D018AC
:103D0600309840E5E92423F5EB30D707E5F904F5CB
:103D1600FB800385F9FBD291AF99C298E537701401
:103D2600BF0520742C2537F582E43469F583EFF05E
:103D36000537800F742C2537F582E43469F583EF57
:103D4600F0053730992BE53CC395365013AE3C054C
:103D56003C742C2EF582E4346AF583E0F599800FE5
:103D6600E53CC395364008053CD296C290C219C2BE
:013D760099B3
:093D7700D0D0D082D083D0E0321C
:102D6F007BFF7A247963121E81906890E07014754E
:102D7F0050FF7551247552BA7BFF7A24797C121E4D
:102D8F008180127550FF7551247552C97BFF7A24CB
:102D9F00797C121E817BFF7A2479D8121E81906A6A
:102DAF004EE0FEA3E0FFC3E49FFFE49EFEAB07FAF5
:102DBF003395E0F9F87F007E8C7D0A7C001222A803
:102DCF008F538E528D518C507BFF7A2479F6121EC1
:102DDF00817BFF7A25792C906891E0F550121E8146
:102DEF00E4906B60F0906B60E0FFC3648094904060
:102DFF0003022E9190689B7420F0E4A3F0EF3395BB
:102E0F00E0FEEF7803C333CE33CED8F9246AF582D0
:102E1F0074263EAF82FE123BF1EF4E6041E4906BA1
:102E2F0062F0124448906B61EFF0643C601BE0FF6E
:102E3F00A3E0FE04F0EEFD3395E0FC749B2DF582CC
:102E4F0074683CF583EFF080D9906B62E0FF3395A7
:102E5F00E0FE749B2FF58274683EF583E4F0906B6F
:102E6F0060E0F55075510175526875539B04F55428
:102E7F007BFF7A257950121E81906B60E004F0027F
:102E8F002DF4906A4CE0FEA3E0FF7C007D0A122136
:0E2E9F00C88E508F517BFF7A25797B121E81E1
:012EAD002202
:0640AE00AB07AA06A905FC
:1040B400E4F540F541AF0119EF60458B828A83E056
:1040C400FDE4FCED5480FEE4EE6240E54030E7168A
:1040D400E54125E0F541E54033F5404341016341C5
:1040E400B263409E800BE54125E0F541E54033F5A0
:1040F40040ED25E0FD0CBC08CA0BBB00010A80B5ED
:0C410400E54090689AF09068EBE541F00F
:01411000228C
:101A1400E4F540F541854182854083E4F00541E5E4
:101A24004170020540B400EDE540B404E8E4906878
:101A340090F07E257F9A123BF1EF4E601B124448D2
:101A44008F48E548B43106906890740AF0E548B4CC
:101A540032069068907464F07E257FA0123BF1EF0B
:101A64004E6023124171A804A905AA06AB077F00A2
:101A74007E8C7D0A7C001222A812233A906A4EEED4
:101A8400F0A3EFF0800A906A4E74FFF0A374B8F0EC
:101A94007E257FA6123BF1EF4E600A1241719068D9
:101AA40091EFF08005E4906891F07E257FAC123BC5
:101AB400F1EF4E6016124171E47B0AFAF9F8122232
:101AC4001D906A4CEEF0A3EFF08009906A4CE4F0AC
:101AD400A37464F0E4F549F543F544F548AF48EFE1
:101AE4003395E0FEEF7803C333CE33CED8F9246ABE
:101AF400F58274263EAF82FE123BF1EF4E70030274
:101B04001E0A1241718F45E5457003021E18E54512
:101B1400B4FF03E4F545854482854383A37405F04B
:101B2400854482854383A3A37464F08544828543FA
:101B340083A3A3A3E4F0E5442404F582E43543F548
:101B440083E4F0E5442405F582E43543F583E54573
:101B5400F0E5442406F582E43543F583E4F0E544F6
:101B64002407F582E43543F5837407F0E54424083B
:101B7400F582E43543F583E4F0E5442409F582E491
:101B84003543F583E4F0E544240AF582E43543F56E
:101B94008374F8F0E544240BF582E43543F583744B
:101BA400A0F0E544240CF582E43543F583E4F0E544
:101BB40044240DF582E43543F583E4F0E544240E32
:101BC400F582E43543F583E4F0E544240FF582E43B
:101BD4003543F583E4F0E5442410F582E43543F518
:101BE40083E4F0E5442403FFE43543FE7D0E124014
:101BF400AE90689AE0FFE5442411F582E43543F59C
:101C040083EFF09068EBE0FFE5442412F582E435BD
:101C140043F583EFF08544828543837412F0E582B3
:101C2400241AF582E43583F583E4F0AA43A9447BBE
:101C3400018B338A34893590001FE5491221A6901F
:101C4400001DE41221A674202544F544E43543F52F
:101C540043906899E004F0124448EF1223961E0A58
:101C6400001E0A211C9C231E0A3C1D32431D4A46A9
:101C74001CBB491CEA501D02511D1A531CD2551D90
:101C8400EE631D4A661D62691D9A701DB6711DD2F0
:101C9400731D7E7500001C5B12444875F008EFA4A8
:101CA40024E2F582E5F03424AF82FE123BF1EF4EDC
:101CB40060A512417180A0AB33E535241BF9E435EE
:101CC40034FA12217B440112219405498089AB33F3
:101CD400E535241BF9E43534FA12217B4402122140
:101CE400940549021C5BAB33E535241BF9E4353418
:101CF400FA12217B44041221940549021C5BAB3384
:101D0400E535241BF9E43534FA12217B4408122109
:101D1400940549021C5BAB33E535241BF9E43534E7
:101D2400FA12217B44101221940549021C5BAB3347
:101D3400E535241BF9E43534FA12217B44201221C1
:101D4400940549021C5BAB33E535241BF9E43534B7
:101D5400FA12217B44401221940549021C5BAB33E7
:101D6400E535241CF9E43534FA12217B44011221AF
:101D74009474032549F549021C5BAB33E535241CF7
:101D8400F9E43534FA12217B4402122194740325B8
:101D940049F549021C5BAB33E535241CF9E43534C1
:101DA400FA12217B440412219474032549F5490253
:101DB4001C5BAB33E535241CF9E43534FA12217B82
:101DC400440812219474032549F549021C5BAB3382
:101DD400E535241CF9E43534FA12217B4410122130
:101DE4009474032549F549021C5BAB33E535241C87
:101DF400F9E43534FA12217B44201221947403252A
:101E040049F549021C5B0548C3E548648094905039
:0A1E140003021AE1E4F543F544FF70
:011E1E0022A1
:10437C00C2A9438902758C48758A4875D90475DBC6
:10438C004875DC4875DD4875DE48E4F5E9F5F9C299
:06439C00D9D28CD2DE2212
:103FE20043AB01C2E8C2EAE4FFEFC454F0F5B1C347
:103FF200EF64809488500575B3D08003E4F5B3E490
:10400200F5B275BCC8F5BDF5BE75BF7875C4FFF5D0
:10401200C5F5C675C778F5A3F5A3F5A3F5A3F5A372
:10402200F5A3F5A3F5A30FBF0EBF906890E0FF259F
:10403200E0F5B475B50C75B66C75A11275AB027569
:08404200C13E75C3FF75C20306
:01404A002253
:1041110075B180E4F5B3F5B28526BCE5275403FFFC
:1041210033333354F8FFE52754E04FFFE528C41338
:1041310054074FF5BDE52833333354F8FFE529C45F
:104141001354074FF5BEE52933333354F8F5BF85D2
:104151002BA3852CA3852DA3852EA3852FA3853085
:10416100A38531A38532A3E52A540F2450F5B32248
:102EAE00E59B541F601B200B15E59B541F90689BE0
:102EBE00F07E257FB27C687D9B7B01122FB6E4F5F8
:102ECE009BE5BA30E008E4F5B375B180F5B2E5CF15
:102EDE00F47003022FB3754A01E4F549E5CFF455BA
:102EEE004A7003022FA1E549C454F0F5B1E5B2547E
:102EFE007F6420706FE5B3540FF52A85BC26E5BDBF
:102F0E00541FFF131313541FFFE5BD54E044184F15
:102F1E00F527E5BDC43354E0FFE5BE131313541F6C
:102F2E004FF528E5BEC43354E0FFE5BF1313135429
:102F3E001F4FF52985A32B85A32C85A32D85A32EA5
:102F4E0085A32F85A33085A33185A332E4F5B2E5A1
:102F5E0026547EB5260575B350800375B3D0E52A89
:102F6E002405FF22E5B2549F6023200B207E257F8F
:102F7E00BD1232B1AFB27E007D0312347FAFB37E8D
:102F8E00007D0312347F7E257FC81232B1E4F5B284
:102F9E0075B3D0E54A25E0F54A0549E549C39408DD
:072FAE005003022EEA7F0030
:012FB50022F9
:1037D600C219E4F537F50BD296F536F53CF524FF1C
:1037E6007F409068ECE4F0A3DFFCE4906897F0A3D8
:1037F600F0FF75F002EFA42490F582E5F03466F54B
:103806008374FFF075F002EFA42491F582E5F0349D
:1038160066F583747FF00FBFFED8E4906897F0A337
:10382600F0F53DF546121A14123FE2C2ADE4F5C9B1
:10383600D2CDD2CCC2C9C2CAF5CDF5CC906A4EE083
:10384600F5CBA3E0F5CA85CBCD85CACCE4F5985374
:1038560087BFD29E438740C29FC2ACC298C29975A9
:10386600B81075B710D2CAD29CD2AC12437CC2D95A
:10387600E5E92464F5EB30D706E5F904F5FB228586
:02388600F9FB4C
:01388800221D
:0100220022BB
:014479002220
:01447A00221F
:01447B00221E
:103EFC00854482854383E07010F543F54485448204
:103F0C00854383E070037F0122E5442401FFE435FF
:103F1C0043F5838F8263A201906A2C63A2017F1404
:103F2C001227C5854482854383E0F536E544454335
:103F3C00700B052453240F906897F0A3F0200B0707
:103F4C007E257FCA1232B1E4F53CD290C291C29662
:103F5C00C2992099FDD299200B0B7E6A7F2CE4FB31
:083F6C00AD3612363C7F002245
:1039C900E546C394404003E4F54674EC2546F58288
:1039D900E43468F583E0FF30E16F74EC2546F58245
:1039E900E43468F583EF54FDF0E4906476F0A37451
:1039F9000DF090667BE0906478F0A37419F0A374DD
:103A090048F0A37479F0E546131313541FFF906827
:103A190091E02F90647CF0E546540725E025E024E9
:103A290080A3F0A37408F0F5F0E546A42490F5828C
:103A3900E5F03466F58363A20190647F63A2017F98
:0E3A4900081227C505467F012205467F002290
:01447C00221D
:10371700E4F538F539853F82853E83E0F53A053F84
:10372700E53F7002053EF582853E83E0F53B053FA8
:10373700E53F7002053E906897E0FEA3E02490F510
:103747008274663EF583E0653A6029906897E0A346
:10375700E0FF2490F58274663EF583E53AF0EF7852
:1037670003CEC313CE13D8F924ECF58274683EF563
:10377700837407F0906898E004F07006906897E00B
:1037870004F0906897E0FEA3E02490F58274663E0B
:10379700F583E0653B6029906897E0A3E0FF2490FC
:1037A700F58274663EF583E53BF0EF7803CEC313ED
:1037B700CE13D8F924ECF58274683EF5837407F0CC
:0F37C700906898E004F07006906897E004F02294
:1042CD00906897E0FEA3E02490F58274663EF58336
:1042DD0074FFF0906898E004F07006906897E00421
:1042ED00F0906897E0FEA3E02490F58274663EF5A9
:1042FD0083747FF0906898E004F07006906897E002
:03430D0004F02297
:100F620074EC253DF582E43468F583E020E0020567
:100F72003DE53DC394404003E4F53D122EAEEF60E3
:100F820069E529640F7063906891E0FF6528705AE3
:100F920074EC253DF582E43468F583E0FE30E04AE6
:100FA20074EC253DF582E43468F583EE54FEF07569
:100FB2002648752779E53D131313541FFEEF2EF5CE
:100FC20028E53D540725E025E02480F529752A0807
:100FD20075F008E53DA42490F582E5F03466F583CA
:100FE2007D2B7F081227BC124111300249C20290A8
:100FF2006893E004F07006906892E004F0D3906881
:1010020093E094B8906892E0940B402AE4F0A3F045
:10101200F54874EC2548F582E43468F583E030E263
:101022000E74EC2548F582E43468F5837407F00504
:1010320048E548B440DC3000469080E8E0700F128A
:10104200404B300D077E257FD01232B1C21D9080F9
:10105200E8E0B40E129080037408F0300D077E258C
:101062007FD91232B1C21D9080E8E0B4060F201D74
:101072000C300D077E257FE41232B1D21DC2002052
:101082001D0302113A2019071235608F488003E4CC
:10109200F548E5486047300D0C7E257FFA7C6A7D75
:1010A20054FB122FB6E5E92410F5EB30D708E5F929
:1010B2002428F5FB8006E5F92427F5FB906A5463A2
:1010C200A201906A2C63A201AF481227C585483657
:1010D200E4F53CD290C291D219C296D29920D9039A
:1010E200021582C2D9E5E92410F5EB30D708E5F9FB
:1010F2002428F5FB8006E5F92427F5FBE537D39490
:10110200005003021582C291853742E4F537906997
:101112002C63A201906A5463A201AF421227C5AFA9
:10112200421231C1200D030215827E257FFF7C6AA7
:101132007D54AB42122FB62220D903021582C2D9A6
:10114200E537D39400500302143AC291853742E442
:10115200F537F50B200B0D7E267F047C697D2C7BF9
:1011620014122FB6753E69753F2E053FE53FAE3E20
:101172007002053E14F5828E83E0646660030215F8
:1011820076053FE53FAE3E7002053E14F5828E8342
:10119200E06003021576E5442405F582E43543F563
:1011A20083E0FF053FE53FAC3E7002053E14F58249
:1011B2008C83E06F6003021576053FE53FAE3E701B
:1011C20002053E14F5828E83E060030215767E6985
:1011D2007F2E7D101240AE9068EBE0FF90689AE09F
:1011E2004F6010300B030215767E267F081232B153
:1011F2000215767E697F3E7D101240AE9068EBE06C
:10120200FF90689AE04F6010300B030215767E263D
:101212007F151232B10215767E697F4E7D10124023
:10122200AE9068EBE0FF90689AE04F6010300B03DD
:101232000215767E267F221232B10215767E697FF2
:101242005E7D101240AE9068EBE0FF90689AE04F2E
:101252006010300B030215767E267F2F1232B10208
:1012620015767E697F6E7D101240AE9068EBE0FFCE
:1012720090689AE04F6010300B030215767E267F4D
:101282003C1232B10215767E697F7E7D101240AE2D
:101292009068EBE0FF90689AE04F6010300B030219
:1012A20015767E267F491232B10215767E697F8ECF
:1012B2007D101240AE9068EBE0FF90689AE04F60BC
:1012C20010300B030215767E267F561232B10215BC
:1012D20076E544241FF582E43543F583E075F00298
:1012E200A4FF906897E5F0F0A3EFF0E544241DF524
:1012F20082E43543F583E4F0E544241BF582E435CA
:1013020043F583E0F54530E009753E69753F821289
:101312003717E54530E109753E69753F8012371789
:10132200E54530E209753E69753F94123717E54588
:1013320030E309753E69753F96123717E54530E48B
:1013420009753E69753F9E123717E54530E5097507
:101352003E69753F66123717E54530E609753E6905
:10136200753F68123717E544241CF582E43543F5CE
:1013720083E0F54530E01B753E69753F3212371741
:10138200753E69753F3A123717753E69753F4412CB
:101392003717E54530E11B753E69753F3412371743
:1013A200753E69753F3E123717753E69753F4612A5
:1013B2003717E54530E21B753E69753F3612371720
:1013C200753E69753F40123717753E69753F481281
:1013D2003717E54530E31B753E69753F38123717FD
:1013E200753E69753F42123717753E69753F4A125D
:1013F2003717E54530E41B753E69753F8E12371786
:10140200753E69753F90123717753E69753F9212A6
:101412003717E54520E50302151C753E69753F60E7
:10142200123717753E69753F62123717753E697537
:101432003F6412371702151CE544241DF582E4357A
:1014420043F583E0D3940A500302150EE544241FAA
:10145200F582E43543F583E075F002A4FF906897C6
:10146200E5F0F0A3EFF0E544241BF582E43543F503
:1014720083E0F54530E0031242CDE54530E1031249
:1014820042CDE54530E2031242CDE54530E3031299
:1014920042CDE54530E4031242CDE54530E5031285
:1014A20042CDE54530E6031242CDE544241CF582E7
:1014B200E43543F583E0F54530E0091242CD1242AE
:1014C200CD1242CDE54530E1091242CD1242CD1294
:1014D20042CDE54530E2091242CD1242CD1242CD53
:1014E200E54530E3091242CD1242CD1242CDE54527
:1014F20030E4091242CD1242CD1242CDE54530E52B
:10150200191242CD1242CD1242CD800EE544241D65
:10151200F582E43543F583E004F0906A4CE0FEA3E3
:10152200E0FF4E6020201B1BE025E9F5EB30D708D9
:10153200EE25F904F5FB8008906A4CE025F9F5FBED
:10154200D21B22C21BE536600B74202544F544E40D
:101552003543F543E5E924E8F5EB30D708E5F9240E
:1015620004F5FB8006E5F92403F5FB123EFCEF705F
:101572000FC21A22200BA37E267F631232B1809AF9
:011582002246
:03001E007F00223E
:103A63000208DFE493A3F8E493A34003F68001F292
:103A730008DFF48029E493A3F85407240CC8C33364
:103A8300C4540F4420C8834004F456800146F6DF33
:103A9300E4800B0102040810204080904472E47E0D
:103AA300019360BCA3FF543F30E509541FFEE49328
:103AB300A360010ECF54C025E060A840B8E493A3EF
:103AC300FAE493A3F8E493A3C8C582C8CAC583CA1A
:103AD300F0A3C8C582C8CAC583CADFE9DEE780BED2
:014478000043
:10217B00BB010689828A83E0225002E722BBFE0262
:09218B00E32289828A83E4932295
:10219400BB010689828A83F0225002F722BBFE012A
:0221A400F32224
:1021A600F8BB010DE58229F582E5833AF583E8F06F
:1021B600225006E92582C8F622BBFE05E92582C81B
:0221C600F22203
:1021C800BC000BBE0029EF8DF084FFADF022E4CCFB
:1021D800F875F008EF2FFFEE33FEEC33FCEE9DECC4
:1021E800984005FCEE9DFE0FD5F0E9E4CEFD22ED0A
:1021F800F8F5F0EE8420D21CFEADF075F008EF2F54
:10220800FFED33FD4007985006D5F0F222C398FD44
:052218000FD5F0EA22E1
:10221D00E88FF0A4CC8BF0A42CFCE98EF0A42CFC60
:10222D008AF0EDA42CFCEA8EF0A4CDA8F08BF0A4DE
:10223D002DCC3825F0FDE98FF0A42CCD35F0FCEB3D
:10224D008EF0A4FEA9F0EB8FF0A4CFC5F02ECD3902
:0F225D00FEE43CFCEAA42DCE35F0FDE43CFC226F
:10226C0075F008758200EF2FFFEE33FECD33CDCC29
:10227C0033CCC58233C5829BED9AEC99E5829840AC
:10228C000CF582EE9BFEED9AFDEC99FC0FD5F0D689
:10229C00E4CEFBE4CDFAE4CCF9A88222B800C1B9B3
:1022AC000059BA002DEC8BF084CFCECDFCE5F0CBF1
:1022BC00F97818EF2FFFEE33FEED33FDEC33FCEB2A
:1022CC0033FB10D703994004EB99FB0FD8E5E4F9E5
:1022DC00FA227818EF2FFFEE33FEED33FDEC33FCD2
:1022EC00C933C910D7059BE99A4007EC9BFCE99AC6
:1022FC00F90FD8E0E4C9FAE4CCFB2275F010EF2F0B
:10230C00FFEE33FEED33FDCC33CCC833C810D7070A
:10231C009BEC9AE899400AED9BFDEC9AFCE899F845
:0E232C000FD5F0DAE4CDFBE4CCFAE4C8F922D8
:0E233A00C3E49FFFE49EFEE49DFDE49CFC22B4
:10234800EB9FF5F0EA9E42F0E99D42F0E89C45F0EB
:012358002262
:0C235900ECF0A3EDF0A3EEF0A3EFF022F7
:10236500A8828583F0D083D08212237C12237C122D
:10237500237C12237CE473E493A3C583C5F0C58352
:10238500C8C582C8F0A3C583C5F0C583C8C582C8C2
:012395002225
:10239600D083D082F8E4937012740193700DA3A3D6
:1023A60093F8740193F5828883E4737402936860EA
:0623B600EFA3A3A380DFEA
:101E1F00E55C2450F8E6055C22784D3017027850C7
:101E2F00E475F0011223E902217B2010EB7F2ED203
:101E3F00108018EF540F2490D43440D4FF30140B7B
:101E4F00EF24BFB41A0050032461FFE55D60021553
:101E5F005D0560E5607002055F30170D784DE47524
:101E6F00F0011223E9EF0221940242847403D21786
:101E7F008003E4C217F55C8B4D8A4E894FE4F55D04
:101E8F00F55FF560E55D60077F20121E5A80F575DE
:101E9F005EFFC211C210C212C213C215C216C218FF
:101EAF00121E28FF700D3017057F00121E6BAF60DA
:101EBF00AE5F22B4255FC2D5C214121E28FF24D0F4
:101ECF00B40A00501A75F00A785D30D50508B6FFD0
:101EDF000106C6A426F620D5047002D21380D92499
:101EEF00CFB41A00EF5004C2E5D21402206BD21106
:101EFF0080C6D21080C0D21280BCD2D580BAD21583
:101F0F0080B47F20121E5A2012077401B55D004065
:101F1F00F1121E1FFF121E5A021E93D218D21680E4
:101F2F0095121E1FFB121E1FFA121E1FF94A4B702D
:101F3F0006793C7A217BFF20122EE55D602A7E0018
:101F4F008E827583001223BC60060EEE655E70F004
:101F5F00C2D5EBC0E0EAC0E0E9C0E0EE1220B2D09B
:101F6F00E0F9D0E0FAD0E0FB12217BFF60AAEBC0D2
:101F7F00E0EAC0E0E9C0E0121E5AD0E02401F9D037
:101F8F00E03400FAD0E0FBE55E0460DCD55ED9807A
:101F9F00877BFF7A2079AED212809C7910800279EC
:101FAF0008C216C2188008D2D5790A8004790AC2ED
:101FBF00D5E55E047002F55EE4FAFDFEFF121E1F0A
:101FCF00FC7B08201113121E1FFD7B1030100A120C
:101FDF001E1FFE121E1FFF7B20EC3382D592D550A1
:101FEF0013C3E43010069FFFE49EFEE42011039D0F
:101FFF00FDE49CFCE4CBF8C211EC700CCFCECDCC41
:10200F00E824F8F870F38017C3EF33FFEE33FEEDDB
:10201F0033FDEC33FCEB33FB994002FB0FD8E9EBBC
:10202F00301105F8D0E0C448B211C0E00AEC4D4EB3
:10203F004F78207B0070C2EAB55E0040BCC0E01252
:10204F0020B4D0F0D0E0201104C4C0E0C4B211C05D
:10205F00F0121E43D0F0D5F0EB021E931223961F01
:10206F0030531FAA581F014C1EFD421FAE4F1FB603
:0F207F00441FB6491F16431FBC551FA0461FA084
:10208E00451FA047215C501F052D1F092E1F2C2B0D
:10209E001F0D231F2A2021452A1EC54800001F247C
:1020AE003F3F3F00790AA2D5201314301509B9100D
:1020BE00020404B9080104A2D5201602500104201E
:1020CE0012689212B55D005034C0E07F20301319B3
:1020DE007F30A21272167215500F12210BC212C24D
:1020EE0016C215C2187F30800F301503E9C0E012FA
:1020FE001E5A301503D0E0F9D0E0B55DCC3015177F
:10210E007F30B9100C121E5A7F583014077F78801A
:10211E0003B90803121E5A3012057F2D021E5A7F74
:10212E00202018F87F2B2016F322921280CF286ED3
:10213E00756C6C2900D211121E1F3011F8C2117865
:10214E005D30D50108F6021EC52D50434958121EAA
:10215E001F2403B405004001E490215793121E4B37
:0D216E00743A121E4BD213755D04021FAAB5
:1028D3008B4A8A4B894CE4F556F555F554F553F577
:1028E30051F552E54E454F454D6012EBC0E0EAC04D
:1028F300E0E9C0E0AB4DAA4EA94F1223F9AB4A055C
:102903004CE54CAA4B7002054B14F912217BF55789
:10291300C394094007E557D3940D40E1E55764207C
:1029230060DBE557B42D054352038016E557B42BFE
:1029330005435201800C74FF254CF54C74FF354B55
:10294300F54BE55060046410703FAB4AAA4BA94CA9
:1029530012217B64306009E550702E75500A80297E
:102963009000011223BCFF64786004EFB458134352
:1029730052017550107402254CF54CE4354BF54B60
:102983008007E5507003755008AB4A054CE54CAA27
:102993004B7002054B14F912217BF557C394614028
:1029A3000AE557D3947A50035357DF74D02557F56C
:1029B30057C3940A400CE5579411406D74F9255799
:1029C300F557E557D39550506043520185565B85C3
:1029D300555A855459855358AF507E00E4FCFDABDE
:1029E30056AA55A954A85312221DC8ECC8C9EDC94B
:1029F300CAEECACBEFCBE4FCFDFEEB2557F556EE52
:102A03003AF555ED39F554EC38F553AF56AE55ADAF
:102A130054FCAB5BAA5AA959A858D31223485003B4
:102A230002298C43520402298CE55220E003E480FE
:102A33002DE54E454F454D601EAB4AE54C24FFF94D
:102A4300E54B34FFFAEBC0E0EAC0E0E9C0E0AB4D90
:102A5300AA4EA94F1223F9E55230E20774FFFFFE95
:102A6300FDFC22E552AF56AE55AD54AC5330E103F5
:042A730002233A22DE
:1023BC00BB010CE58229F582E5833AF583E02250D6
:1023CC0006E92582F8E622BBFE06E92582F8E22220
:0D23DC00E58229F582E5833AF583E493223A
:1023E900FAE6FB0808E6F925F0F618E6CA3AF622F5
:1023F900BB011A89828A83D0F0D0E0F8D0E0F9D005
:10240900E0FAD0E0FBE8C0E0C0F00224515016E940
:10241900F8D083D082D0E0F9D0E0FAD0E0FBC082D6
:10242900C083022448BBFE16E9F8D083D082D0E0ED
:0F243900F9D0E0FAD0E0FBC082C08302245A221F
:09244800EBF608EAF608E9F622B9
:09245100EBF0A3EAF0A3E9F0228C
:09245A00EBF208EAF208E9F222B3
:00000001FF
